:0300330002001AAE
:04001A0053D8EF3296
:100003008E568F57E5571557AE56700215564E60EC
:0700130005120FA280EE228E
:0300230002004692
:10004600C0E0C083C082C086758600C0D075D00867
:1000560030990E300B07A20E929B853699C299D223
:10006600122012030202F9C2123003197E7E7F406B
:10007600751A7E751B407517007E7D7FC075187DCD
:100086007519C080177E7D7FC0751A7D751BC0757A
:1000960017017E7E7F4075187E751940200B03027E
:1000A6000184E53AC39553503C200C342009319025
:1000B6007F9BE055387029301012AF3A053AE51BA0
:1000C6002FF582E4351AF583E013920EAF3A053A1E
:1000D600E51B2FF582E4351AF583E0F5360202F7C3
:1000E600C20B0202F7300311907FC7E4F0A3E0547D
:1000F60002F51DA3E0F51C8011907FC9E4F0907F06
:03004300020F00A9
:03000000020026D5
:0C002600787FE4F6D8FD75815A020A3399
:40010600C6E05402F51DA3E0F51CE51724FF9203300D0DC20D907FBB7401F0C20B0202F7E51D6005C20B0202F7851C53851982851883E013920D7512FF200C3A2009379082
:400146007F9BE05538702F30101C851982851883A3E013920E851982851883A3A3E0F536753A030202F7753A02851982851883A3E0F5360202F7753A01C20B0202F73003FE
:400186000E907FC6E05402F51DA3E0F51C800C907FC8E05402F51DA3E0F51CE53AC395535003020268E51D6007C214C2050202F7851C53851B82851A83E013920D7512FF61
:4001C600300C03020260300903020260907F9BE05538600302026030101B851B82851A83A3E013929B851B82851A83A3A3E0F599753A03800D851B82851A83A3E0F5997575
:400206003A02E53AC395534026300307907FC7E4F08005907FC9E4F0E51724FF9203200D030202F7C20D907FBB7401F00202F7301012AF3A053AE51B2FF582E4351AF58394
:40024600E013920EAF3A053AE51B2FF582E4351AF583E0F536D20B0202F7753A01C2140202F7300C030202F53009030202F5907F9BE055387079301012AF3A053AE51B2FF2
:40028600F582E4351AF583E013929BAF3A053AE51B2FF582E4351AF583E0F599E53AC395534022300307907FC7E4F08005907FC9E4F0E51724FF9203300D36C20D907FBB0E
:4002C6007401F0802C301012AF3A053AE51B2FF582E4351AF583E013920EAF3A053AE51B2FF582E4351AF583E0F536D20B8002C214D201209803020435C298200203020383
:40030600A2201527AF39053974802FF582E4347EF583E599F030104DAF39053974802FF582E4347EF583E598F0803A859955E555B54704D209802EE555B54604C20980251C
:40034600AF39053974802FF582E4347EF583E555F0301011AF39053974802FF582E4347EF583E598F0D20FE539C395435003020433907FB8E030E116E539C39440500302F5
:40038600043315391539052B433401020433907FB7E539F0753900C202020433201527AF39053974002FF582E4347EF583E599F030104DAF39053974002FF582E4347EF594
:4003C60083E598F0803A859955E555B54704D209802EE555B54604C2098025AF39053974002FF582E4347EF583E555F0301011AF39053974002FF582E4347EF583E598F0EA
:40040600D20FE539C395434024907FB6E030E112E539C39440401615391539052B433401800B907FB9E539F0753900D202D201300105C201020056D0D0D086D082D083D02F
:40044600E032907FBCE020E154E5346050E531704CE53430E10BE4F52F753401753102800EA208E433F52FC208E4F534753110E4F5567E007B0074242556F9EE3400FA12D8
:400486000C79FF74002556F582E4347DF583EFF00556E556B40CDB907FBD740CF0907FCAE030E1030205D1E4F55674402556F582E4347DF583E0FFE5567C007B00243BF903
:4004C600EC3400FAEF120C920556E556B418DBE53B601175C92075C836853CCA853DCBE4907F9FF0E53E139210929F853F38E540139215E5416009907F98E054FBF0800744
:40050600907F98E04404F0E5426009907F98E0547FF08007907F98E04480F0E548600BC20CC209907F95E04402F0E549600CD209433401907F95E04402F0E54A600DC2AFBB
:40054600C20BD200E4F553F53AD2AFE54B6005301502D209E54C6015907F95E054FDF0907F9EE04402F0907F98E054FDF0E54D600AD29CC298752C0175311EE54E6007C227
:400586009CE4F539F52CE54F6003E4F539E5506002D207E551600AE54D7002F531E5514234E552601F907FD77411F07431F07412F07432F07413F07433F07414F07434F067
:4005C600D203D202D208E4907FCBF0A20CE433FF652960058F29433401A209E433FF652A60058F2A433401907F9BE0FF54086408F55765256006855725433401EF5410643A
:4006060010F55765266006855726433401EF54406440F55765276006855727433401EF54206420F55765286006855728433401907F9AE054406440F557652E600685572E5B
:40064600433401300735C2AF300218907FB8E020E127E5396009907FB7F0E4F539C202C2078016907FB6E020E10FE5396009907FB9F0E4F539D202C207D2AF20053D3003DB
:400686001E907FC6E020E133907E40E013920D753A01907FC7E0F553D2057512FF801C907FC8E020E115907DC0E013920D753A01907FC9E0F553D2057512FF2014332000E6
:4006C60006E53A6553702A30051A300309E4907FC7F0C2038007E4907FC9F0D203C205E4F553F53A300D0AC20DC200907FBB7401F03014030207BF2005030207BF300C0314
:400706000207BF3009030207BF907F9BE0553860030207BF30030C7E7E7F4075587E755940800A7E7D7FC075587D7559C0301012AF3A053AE5592FF582E43558F583E0137C
:40074600921AAF3A053AE5592FF582E43558F583E0F557E53AC39553502A301012AF3A053AE5592FF582E43558F583E013920EAF3A053AE5592FF582E43558F583E0F53688
:40078600D20B8015C20B300309E4907FC7F0C2038007E4907FC9F0D203301004A21A929BD214C2AF855799200B0D300D0AC20DC200907FBB7401F0D2AF22907FE9E0120C70
:4007C600A4091C0009890109E60307E306090D0809010908E90A08F80B00000A24907FEBE024FE601C14700302087924026003020A24740D907FD4F07487907FD5F0020AE6
:400806002B907FEAE0B401047F0280027F037582D875830DEFF07582D175830DF07582CA75830DF07582C375830DF0907FEAE00475829E75830DF0907FEFE0FE907FEEE07B
:400846007C002400F55AEC3EF55975150D75169975829B75830DE0751300F514D3E514955AE51395594006855913855A14120BBA020A2B907FEAE0700B7556FF75570D7503
:4008860058DC802D907FEAE0B4010B7556FF75570D7558E0801B907FEAE0B4020B7556FF75570D7558F080097556FF75570E75581E907FEEE0755900F55AAE57AF588E1512
:4008C6008F168F828E83E0FEA3E08E13F514D3955AE51395594006855913855A14120BBA020A2B907F00E511F0907FB57401F0020A2B907FEAE0F511020A2B120C24907F84
:40090600EAE0F510020A2B907F00E510F0907FB57401F0020A2B907FE8E0247F602714603424026003020A24A216E433FF25E0FFA218E4334F907F00F0E4A3F0907FB57455
:4009460002F0020A2BE4907F00F0A3F0907FB57402F0020A2B907FECE0F45480FFC4540FFFE054072F25E024B4F582E4347FF583E054FD907F00F0E4A3F0907FB57402F00B
:40098600020A2B907FE8E024FE601724026003020A2B907FEAE064016003020A24C216020A2B907FEAE07076907FECE0F45480FFC4540FFFE054072F25E024B4F582E4348D
:4009C6007FF583E4F0907FECE05480FF131313541FFFE054072F907FD7F0E04420F08045907FE8E024FE601024027039907FEAE06401702AD216802D907FEAE07020907F77
:400A0600ECE0F45480FFC4540FFFE054072F25E024B4F582E4347FF5837401F08007907FB4E04401F0907FB4E04402F022C210E4F510F534C209C20CC20BC214C20DC215A5
:400A4600C211C207C212C20FC208F535F539F553F53AF533F530F52FF52EF52DF52CF52BF52AF529F528F527F526F525F524C205C217C219C216C218C204D213C206C20178
:400A8600907F92E054FDF0D2E843D820907FDE7401F0907FDFF0907FAB74FFF0907FA9F0907FAAF05391EF907FAFE04401F0907FAEE0440FF0907FAC740EF0D2AFD2BCD247
:400AC6001A120F7DC21730040312044830042A300627C206E51260161512907FD8E030E6047F0080027F20907F96EFF08006907F967420F0120B1480CD301707C217120741
:400B0600C080C33019C0C219120EDC80B922E53160021531E53960556535704BE533F460020533E533C395444043C2AF30021B907FB8E020E12D907FB7E539F0C202E4F5AA
:400B460039F533F5357512FF8019907FB6E020E112907FB9E539F0D202E4F539F533F5357512FFD2AF8006853935E4F533E52C6030200F07907F9BE030E00FE52D6006E497
:400B8600F52D433401E4F5308014E530D39545500DE530B54506752D014334010530C20F22907FD9E030E2047F0080027F20907F96EFF022E51445136057AE13AF14D3EF0F
:400BC6009440EE940040047E007F40C3E5149FF514E5139EF513E4FDEDC39FE49E501F851682851583E0FC74002DF582E4347FF583ECF00D0516E5167002051580DA907FC4
:400C0600A97401F0907FACE04401F0907FB5EFF022907FACE054FEF0E4907FB5F022E4907F93F0907F9C7430F0907F967420F0907F947401F0907F9D74FFF0907F977486DF
:400C4600F0907F957403F0907F9E7484F0907F98F0E4907FC7F0907FC9F0907FCBF075984043A810907FDE741FF0907FDF740FF0D20422BB010689828A83E0225002E722C3
:400C8600BBFE02E32289828A83E49322BB010689828A83F0225002F722BBFE01F322D083D082F8E4937012740193700DA3A393F8740193F5828883E4737402936860EFA367
:400CC600A3A380DFE4907F95F0907F94F0907F93F0907F9DE04402F0907F97E04442F0907F9C7410F0E4907F96F0907F9D74BEF03016047F8080027F00907F97EFF0E49045
:400D06007F95F0907F9EF0907F98F022C0E0C0F0C083C082C085C084C086758600C0D075D0085391EF907FA97401F0120BBAD0D0D086D084D085D082D083D0F0D0E032C06A
:400D4600E0C083C082C085C084C086758600907FC4E4F05391EF907FAB7404F0D086D084D085D082D083D0E03200000000000000000000000000000000000000000000001C
:400D86000012011001FFFFFF40CD061C010100010200020902430001010080320904000007FF00000007050102400000070502024000000705030240000007058102400002
:400DC600010705820240000107058302400001070584024000010403090410034B00650079007300700061006E002E034B00650079007300700061006E00200055005000A3
:400E0600530048003100310032002D00530065007200690061006C0022035500530041002D003500330020003200300030003200610070007200320036000000C0E0C083DB
:400E4600C082C085C084C0867586005391EF907FAB7402F0D206D086D084D085D082D083D0E032C0E0C083C082C085C084C086758600D2175391EF907FAB7401F0D086D01F
:400E860084D085D082D083D0E032C0E0C083C082C085C084C086758600D2195391EF907FAB7408F0D086D084D085D082D083D0E032C0E0C083C082C085C084C08675860084
:400EC6005391EF907FA97402F0D086D084D085D082D083D0E032120CCA120FB3907FD6E030E712E04401F07F0D7E00120003907FD6E054FEF0120C242200020E6900020EA3
:400F06004200020D4500020E9000020F1000020F1400020D1200020F1C00020EB700020F2400020F3300020F2C00020F58C0E0C083C082C085C084C0867586005391EF90A9
:400F46007FA97404F0D086D084D085D082D083D0E032C0E0C083C082C085C084C0867586005391EF907FA97408F0D086D084D085D082D083D0E032907FD6E054FBF0E044C1
:3D0F860008F0301A04E04402F07FF47E01120003907FD6E054F7F0E04404F0227400F58690FDA57C05A3E582458370F922907FD6E04480F04387010000000000222C
:00000001FF
